:020000002429B1
:10000600243083120313FD00FD0B072800000800AF
:1000160083120313F801F9011030FC00710DF80D7D
:10002600F90D7408F8027508031C750FF902031818
:1000360023287408F80775080318750FF9070310C5
:0A004600F00DF10DFC0B112808006D
:0E005000831203133F088A003E088200080056
:10005E0028208A110A128000840ABE0A0319BF0AD8
:08006E00F003031D2F28080018
:10007600C330831203139F0540309F05F03083166B
:100086009F0483129F174408F000F00D7010F00DC6
:10009600701070089F041F1403209F149F1C55287E
:1000A600000051281F101E08F100F00183161E08DB
:0800B600F0040030F104080021
:1000BE0083120313FB01FA01F9018030F800F10CF1
:1000CE00F00C031C73287408F90775080318750FD4
:1000DE00FA070318FB0A0310F01F7B287408FA07AF
:1000EE0075080318750FFB07FB0CFA0CF90CF80CCE
:1000FE00031C66287B08F3007A08F2007908F100E9
:06010E007808F000080073
:10011400103083120313F4002730F5003908F0007F
:100124003A08F1000B207008BD00E830F4000330F9
:10013400F5003908F0003A08F1000B200A30F40009
:100144000030F5000B207808F0007908F100700801
:10015400B8006430F4000030F5003908F0003A08C3
:10016400F1000B200A30F4000030F5000B20780871
:10017400F0007908F1007008BC000A30F400003087
:10018400F5003908F0003A08F1000B200A30F400B9
:100194000030F5000B207808F0007908F1007008B1
:1001A400BB002D08003A031DDA283D08AC00EE28F8
:1001B4002D08013A031DE1283808AC00EE282D086B
:1001C400023A031DE8283C08AC00EE282D08033A47
:1001D400031DEE283B08AC002D08013A031DF82846
:1001E4002C082E3E84000008C300FD282C08203E65
:1001F40084000008C3002D08003A031D0629EF30CF
:10020400C0000130AD001F292D08013A031D0F293C
:10021400DF30C0000230AD001F292D08023A031D53
:100224001829BF30C0000330AD001F292D08033A40
:10023400031D1F297F30C000AD014008860043081C
:040244008700080027
:10024800C03083120313A000F930A100A430A2002B
:10025800B030A3009930A4009230A5008230A600E7
:10026800F830A7008030A8009830A900AA01AB0197
:10027800AC01AD014030AE007930AF002430B000A1
:100288003030B1001930B2001230B3000230B4007F
:100298007830B500B6011830B700013003179E005A
:1002A8009F0199019A01FF308316031385000F30CF
:1002B800860087018030810083128101A0308B0085
:1002C800B901BA0101309F0083169F018A20AA0A4A
:1002D8000319AB0A2B08003C031D74292A08323C79
:1002E80003188829C4013B2070088312C1007108D3
:1002F800C2003130F4000030F5005F207008B9000A
:0C0308007108BA00AA01AB016A2989291A
:02400E00D400DC
:00000001FF
